:100000000C945A000C9475000C9475000C947500B7
:100010000C9475000C9475000C9475000C9475008C
:100020000C9475000C9475000C9475000C9475007C
:100030000C9475000C9475000C9475000C9475006C
:100040000C94A6050C9475000C9475000C94750026
:100050000C9475000C9475000C9475000C9475004C
:100060000C9475000C94750000000007000201005C
:100070000003040600000000000000000102040864
:100080001020408001020408102001020408102002
:10009000040404040404040402020202020203032E
:1000A000030303030000232629000025282B00005A
:1000B00024272A0011241FBECFEFD4E0DEBFCDBF1E
:1000C00011E0A0E0B1E0EEE9FEE002C005900D9283
:1000D000AA35B107D9F711E0AAE5B1E001C01D9238
:1000E000A238B107E1F70C949B050C940000FF9235
:1000F0000F931F93CF93DF93EC018B01FF24672BAA
:1001000011F481E0F82E6F2D8C2F0E94BB0661E068
:1001100070E080E090E00E94E305602F8C2F0E9449
:10012000BB0661E070E080E090E00E94E3056F2D87
:100130008C2F0E94BB0661E070E080E090E00E949E
:10014000E305DF91CF911F910F91FF900895EF92FA
:10015000FF920F931F93CF93DF937C018C0154E0A8
:10016000159507955A95E1F7C0914501D091460143
:1001700008C0602F61708C2F0E94BB0615950795F3
:10018000219680914101909142018C179D078CF737
:1001900061E070E080914D0190914E010E947700E6
:1001A00061E070E080E090E00E94E305C0914501CD
:1001B000D091460108C06E2D61708C2F0E94BB0645
:1001C000F594E794219680914B0190914C018C1706
:1001D0009D078CF7870124E0159507952A95E1F78F
:1001E000C0914301D091440108C0602F61708C2FF1
:1001F0000E94BB061595079521968091410190912B
:1002000042018C179D078CF761E070E080914D01F1
:1002100090914E010E947700DF91CF911F910F9135
:10022000FF90EF900895EF92FF920F931F93CF935B
:10023000DF937C0161E0809141010E94BB0660E098
:10024000809143010E94BB068701E4E01595079564
:10025000EA95E1F7C0914501D091460108C0602FB1
:1002600061708C2F0E94BB06159507952196809191
:100270004B0190914C018C179D078CF761E070E069
:1002800080914D0190914E010E94770061E070E0F5
:1002900080E090E00E94E30561E0809141010E94CE
:1002A000BB0660E0809143010E94BB06C0914501FE
:1002B000D091460108C06E2D61708C2F0E94BB0644
:1002C000F594E794219680914B0190914C018C1705
:1002D0009D078CF761E070E080914D0190914E0197
:1002E0000E947700DF91CF911F910F91FF90EF90C7
:1002F00008950F931F93CF93DF939C0164E670E002
:100300000E94060784E690E0AC01649FC001659FEF
:10031000900D749F900D11248901081B190BC801C1
:100320006AE070E00E940607EB016115710529F093
:10033000CB01805D9D4F0E94A7008AE090E09C0168
:10034000C29FC001C39F900DD29F900D1124081B26
:10035000190BC801805D9D4F0E94A700DF91CF91CE
:100360001F910F9108950F931F938C0182E090E0ED
:100370000E94A70064E070E080E090E00E94E30546
:100380000130110521F480EC90E00E94A70061E0AB
:1003900070E080E090E00E94E3051F910F910895C6
:1003A00081E090E00E94A70064E070E080E090E0CF
:1003B0000E94E3050895CF93DF93C0914D01D09142
:1003C0004E0105C061E08C2F0E9454062196809159
:1003D0004101909142018C179D07A4F783E090E0C2
:1003E0000E94A70060E470E080E090E00E94E305D6
:1003F00083E090E00E94A70062E370E080E090E07C
:100400000E94E30583E090E00E94A70062E370E0B1
:1004100080E090E00E94E30582E090E00E94A70067
:1004200062E370E080E090E00E94E3058CE290E0FF
:100430000E94A70064E170E080E090E00E94E30584
:1004400086E090E00E94A70064E170E080E090E028
:100450000E94E3058CE090E00E94A70064E170E058
:1004600080E090E00E94E30581E090E00E94A70018
:1004700064E670E080E090E00E94E30580E890E0B0
:100480000E94A7006EE170E080E090E00E94E3052A
:10049000DF91CF91089560E0809151010E94540650
:1004A00061E0809151010E94BB0660E080914F01A4
:1004B0000E94540661E080914F010E94BB0608959E
:1004C00060E080917C010E94540661E080917C0193
:1004D0000E94BB0660E0809157010E94540661E0D3
:1004E000809157010E94BB0660E0809153010E94F9
:1004F000540661E0809153010E94BB06089561E0BB
:1005000080913F010E94540661E080913F010E946A
:10051000BB060E94DB010E944B020E94600208950C
:100520008091780190917901892BA1F480915E01ED
:1005300090915F012091620130916301892B19F440
:100540002F5F3F4F02C0245C3F4F309363012093E5
:100550006201089580916001909161012091640190
:1005600030916501892B19F42F5F3F4F02C0245C45
:100570003F4F3093650120936401209164013091D5
:10058000650180916201909163018217930724F4C1
:1005900030936301209362010895809178019091D6
:1005A0007901892BA1F480915E0190915F012091E6
:1005B000620130916301892B19F42150304002C04F
:1005C0002C53304030936301209362010895809151
:1005D0006001909161012091640130916501892B46
:1005E00019F42150304002C02C5330403093650143
:1005F000209364010895809151010E9472069C012C
:1006000090935B0180935A0180915C0190915D0110
:10061000892B09F04BC02130310509F047C080918A
:100620004F010E947206892B19F40E94CD0202C06C
:100630000E949002809162019091630197FF04C033
:1006400010926301109262018091640190916501A2
:1006500097FF04C0109265011092640180916201BD
:1006600090916301CC973CF081E090E090935F0122
:1006700080935E0104C010925F0110925E01809130
:10068000640190916501CC973CF081E090E09093FB
:1006900061018093600104C01092610110926001B9
:1006A00081E090E090933C0180933B0180915A015E
:1006B00090915B0190935D0180935C0108950E948D
:1006C000CB0520916E0130916F01409170015091E6
:1006D0007101621B730B840B950B6C52714080404F
:1006E000904058F40E94CB0560936E0170936F01A7
:1006F000809370019093710108950E94CB056093DF
:100700006E0170936F0180937001909371018091DD
:100710007A0190917B01019690937B0180937A01FD
:10072000049724F010927B0110927A0180917A0153
:1007300090917B018130910529F490937901809308
:10074000780104C0109279011092780181E090E064
:1007500090933E0180933D01089580917A0190919C
:100760007B010297B1F50E94CB0520916A0130917F
:100770006B0140916C0150916D01621B730B840BF6
:10078000950B6C5271408040904058F40E94CB050C
:1007900060936A0170936B0180936C0190936D017B
:1007A00008950E94CB0560936A0170936B0180935A
:1007B0006C0190936D0120E030E080917801909180
:1007C0007901892B11F421E030E0309379012093F5
:1007D000780181E090E090933C0180933B01089583
:1007E0000E94CB05209172013091730140917401F8
:1007F00050917501621B730B840B950B6C52714009
:100800008040904058F40E94CB0560937201709331
:100810007301809374019093750108950E94CB0534
:1008200060937201709373018093740190937501CA
:1008300020E030E08091760190917701892B11F4CE
:1008400021E030E030937701209376010895672B03
:1008500029F40E94790182E290E009C06CE370E023
:100860000E940607CB010E94790187E290E00E9476
:10087000130108959C01672B29F06CE370E00E943E
:1008800006079B01C90164E670E00E94060784E642
:1008900090E0AC01649FC001659F900D749F900D26
:1008A0001124281B390BC9016AE070E00E94060779
:1008B000672B19F083E090E0089582E090E00895BE
:1008C0000F931F93CF93DF9380913D0190913E0151
:1008D000892B81F180E090E00E94B301C0E0D0E07C
:1008E00006C0992787FD90950E9413012196E091FB
:1008F0007A01F0917B01EE0FFF1FED5CFE4F01903E
:10090000F081E02DEC0FFD1F8081882351F705C099
:1009100080E292E00E9413012196C031D105C4F318
:1009200010923E0110923D0181E090E090933C01D5
:1009300080933B0180913B0190913C01892B09F40C
:100940005FC081E090E00E94B30180917A019091B4
:100950007B01019729F400E010E0C1E0D0E021C064
:1009600060915E0170915F018091620190916301DD
:100970000E942704C0917A01D0917B01C130D1053A
:1009800019F400E010E00DC060915E0170915F010C
:1009900080916201909163010E943A048C0120973A
:1009A00071F0239761F06091600170916101809115
:1009B0006401909165010E943A04080F191FC0E17B
:1009C000D0E005C080E290E00E94130121970C174F
:1009D0001D07C4F380917A0190917B01009761F02B
:1009E000039751F060916001709161018091640101
:1009F000909165010E94270410923C0110923B01E6
:100A000080917C010E947206892B11F40E94F003F0
:100A10008091760190917701892B09F475C08091BE
:100A20007A0190917B01039709F480C00E94CB0565
:100A30009B01AC018091660190916701A0916801D2
:100A4000B0916901281B390B4A0B5B0B6091620165
:100A50007091630180917A0190917B01892B31F033
:100A60008091640190916501681B790BC8EED3E019
:100A70006C9FC0016D9F900D7C9F900D1124AA2743
:100A800097FDA095BA2F82179307A407B50708F022
:100A90004DC060E080913F010E94BB0680917A01C9
:100AA00090917B01892B29F464E670E080E090E06E
:100AB0000FC080916401909165018C9FB0018D9F62
:100AC000700D9C9F700D1124882777FD8095982FBD
:100AD0000E94E30561E080913F010E94BB060E94F5
:100AE000CB056093660170936701809368019093D2
:100AF000690180917A0190917B010197B9F410927C
:100B000077011092760112C00E94FB02809157017A
:100B10000E947206892B11F40E945F038091530199
:100B20000E947206892B11F40E94AD03DF91CF91D0
:100B30001F910F910895CFEFD4E0DEBFCDBF0E948B
:100B400012060E947F020E946004FDCF1F920F9246
:100B50000FB60F9211248F939F93AF93BF93809101
:100B60007E0190917F01A0918001B0918101019659
:100B7000A11DB11D80937E0190937F01A093800100
:100B8000B0938101BF91AF919F918F910F900FBE54
:100B90000F901F90189560917E0170917F01809158
:100BA00080019091810127E0660F771F881F991FB0
:100BB0002A95D1F72DE730E040E050E00E94190778
:100BC000CA01B9010895AF92BF92CF92DF92EF921E
:100BD000FF920F931F935B016C010E94CB057B0179
:100BE0008C010E94CB056E197F09800B910B6A1551
:100BF0007B058C059D05A8F31F910F91FF90EF9049
:100C0000DF90CF90BF90AF900895019751F0880F7B
:100C1000991F880F991F02972FB7F8940197F1F742
:100C20002FBF0895789410927E0110927F01109248
:100C300080011092810184B5826084BD84B5816099
:100C400084BD85B5826085BD85B5816085BDEEE6D4
:100C5000F0E0808181608083E1E8F0E08081826063
:100C60008083808181608083E0E8F0E08081816022
:100C70008083E1EBF0E0808184608083E0EBF0E052
:100C8000808181608083EAE7F0E0808184608083F6
:100C900080818260808380818160808380818068A0
:100CA00080831092C1000895282F3327C9018458EA
:100CB0009F4FFC01949120573F4FF9018491882365
:100CC00081F0E82FFF27E255FF4FE491FF276623CD
:100CD00029F4808190958923808308958081892BD0
:100CE00080830895482F5527CA0188599F4FFC01DA
:100CF0002491CA0184589F4FFC01949140575F4F43
:100D0000FA0134913323A1F1222331F1233021F46C
:100D1000809180008F7705C0243031F4809180006D
:100D20008F7D8093800018C0213019F484B58F77AF
:100D300004C0223021F484B58F7D84BD0DC02630DF
:100D400021F48091B0008F7705C0273029F480917D
:100D5000B0008F7D8093B000E32FFF27EC55FF4F4D
:100D6000E491FF278081892319F081E090E00895C4
:100D700080E090E00895482F5527CA0188599F4F79
:100D8000FC012491CA0184589F4FFC019491405763
:100D90005F4FFA0134913323C1F1222331F1233023
:100DA00021F4809180008F7705C0243031F4809148
:100DB00080008F7D8093800018C0213019F484B5A5
:100DC0008F7704C0223021F484B58F7D84BD0DC09F
:100DD000263021F48091B0008F7705C0273029F4A8
:100DE0008091B0008F7D8093B000E32FFF27E755FF
:100DF000FF4FE491FF27662329F480819095892392
:100E0000808308958081892B8083089597FB092E24
:100E100007260AD077FD04D02ED006D000201AF481
:100E2000709561957F4F0895F6F7909581959F4F46
:100E30000895A1E21A2EAA1BBB1BFD010DC0AA1F1B
:100E4000BB1FEE1FFF1FA217B307E407F50720F033
:100E5000A21BB30BE40BF50B661F771F881F991FAE
:100E60001A9469F760957095809590959B01AC01F7
:100E7000BD01CF010895AA1BBB1B51E107C0AA1FEA
:100E8000BB1FA617B70710F0A61BB70B881F991F2B
:0E0E90005A95A9F780959095BC01CD01089563
:100E9E00496E74657276616C00202020202020201F
:100EAE00202020202042756C6200496E7465727697
:100EBE00616C2020202042756C6200547269676755
:100ECE00657200000109011A012B01010001000DDC
:100EDE00000C000B000700080009000A00060005C0
:0A0EEE0000040003000200010000F0
:00000001FF
